:100000000C9404030C941F030C941F030C941F0303
:100010000C941F030C941F030C9474130C941F0373
:100020000C941F030C941F030C941F030C941F03C8
:100030000C942E140C941F030C941F030C941F0398
:100040000C941F030C945E060C941F030C941F0366
:100050000C941F030672652C0375223B59781EBA57
:10006000E07A633BF47C75FF4E7E3172117F0000B5
:10007000000005813504F483200001836246328349
:10008000200000816246307F0000000582778C4F9F
:1000900081432CE28217BF2483A48DD981E1D8A1AA
:1000A00080DB67820502ED0C010510640C05050478
:1000B000830D100501630CFF0103640C050110EDB5
:1000C0000C010104830D1001021C0D020203ED0C52
:1000D0000102101C0D020204830D100202920C0397
:1000E00003031C0D020310920C030304830D100381
:1000F000025E0D0403015D0CFF0403920C03041067
:100100005E0D040404830D101001640C051004CB73
:100110000E201002880D181803830D101801640CAE
:10012000051804210F2D1802B10D171703880D189B
:100130001701640C051704C80F271702DA0D1111F7
:1001400003B10D171101640C051104661021110291
:100150000B0E121203DA0D111201640C0512041AAF
:10016000112412023C0E1515030B0E121501640C1E
:10017000051504630CFF15025C0E161601640C05D0
:1001800016033C0E151604C2112C2001830D1020FD
:1001900002DE0E202003E30E202004E80E202D01B5
:1001A000880D182D023E0FFF2D03430FFF2D045124
:1001B0000F2E2E01880D182E02740FFF2E03790FBB
:1001C000FF2E04870F2F2F01880D182F02AA0FFF73
:1001D0002F03AF0FFF2F04B40F2D2701B10D1727E9
:1001E00002E50FFF2703EA0FFF2704F80F28280175
:1001F000B10D1728021B10FF28032010FF28042E22
:1002000010292901B10D1729024710FF29034C10AD
:10021000FF29045110272101DA0D1121028510FF59
:1002200021038A10FF21049B10222201DA0D1122E2
:1002300002C010FF2203C510FF2204D610232301A1
:10024000DA0D112302FB10FF23030011FF23040525
:10025000112124010B0E1224023911FF24033E1137
:10026000FF24044F112525010B0E1225026811FFF2
:1002700025036D11FF25047E112626010B0E122683
:1002800002A311FF2603A811FF2604AD11242C019F
:100290005C0E162C02E111FF2C03E611FF2C04EB7F
:1002A000111603015D0CFF000000000048033D0330
:1002B0002F0321031303D702D302CB02BE024865EA
:1002C000697A756E672026204257004865697A75FD
:1002D0006E67004257200041757300C303B303A249
:1002E0000392038503750369035D035003C303E1B0
:1002F00003D203CD031E04CA03FB03E8031E04D686
:10030000030604E8031E04FB030604F1031E04169F
:10031000040B044E6F726D616C2F4E6F726D616CC9
:10032000004E6F726D616C2F416273656E6B0041A0
:100330006273656E6B2F416273656E6B00417573FE
:100340002F416273656E6B004175732F41757300A9
:100350004F656C6272656E6E65723A200048656921
:100360007A70756D70653A2000486F6C7A70756DA3
:1003700070653A2000537065696368657270756DC9
:1003800070653A2000536F6C617270756D70653ADC
:1003900020004D69736368657220616B7469763AF9
:1003A00020004D697363686572206175662F7A75E8
:1003B0003A20004B657373656C6D69736368657291
:1003C0003A2000467265693A20004F4B00486F6C36
:1003D0007A004F656C00425720566F7272616E67EB
:1003E0000050756666657200456E657267696521C5
:1003F000004E6163686C61756620004175666865D2
:10040000697A656E200045696E200041626B7565F2
:10041000686C656E20004272656E6E7420004175D6
:100420007320005374617475733A20002A2A2A20BD
:100430005374617274766F7267616E672E2E2E0030
:10044000425241554348574153534552564F5252D9
:10045000414E47004845495A4752454E5A450A20A1
:100460004E6F726D616C626574722E3A0A20416241
:1004700073656E6B626574722E3A004F454C2D4267
:1004800052454E4E45520A20426574726965623A81
:100490000A20566F6E3A0A204269733A004845496D
:1004A0005A554E470A20426574726965623A0A20BD
:1004B000566F6E3A0A204269733A005241554D54C4
:1004C000454D504552415455520A205261756D7444
:1004D000656D702E20313A0A205261756D74656D1C
:1004E000702E20323A0A204E69766561753A0048CE
:1004F00045495A4B555256450A204578706F6E65EE
:100500006E743A0A204D61782E20566F726C6175B8
:10051000663A0A204D696E2E2041757373656E3AF6
:1005200000534552564943454D454E554500535499
:10053000415455530A204272617563687761737341
:1005400065723A0A204865697A756E673A0A2051E1
:1005500075656C6C653A004F454C4B455353454CA3
:100560000A20566F726C61756620203A0A20527517
:1005700065636B6C6175663A0A20537461747573B8
:100580003A00484F4C5A4B455353454C0A20566F3E
:10059000726C61756620203A0A20527565636B6C37
:1005A0006175663A0A205374617475733A00484560
:1005B000495A554E470A20566F726C617566202065
:1005C0003A0A20527565636B6C6175663A0A20536E
:1005D0006F6C6C3A202020202020204175737365B9
:1005E0006E3A004252415543485741535345520ACF
:1005F000204F62656E203A0A20556E74656E3A0A85
:1006000020536F6C61723A0011241FBECFE5D4E015
:10061000DEBFCDBF10E0A0E6B0E0E8EBF3E302C040
:1006200005900D92AA38B107D9F711E0AAE8B0E019
:1006300001C01D92A23AB107E1F70C941E0C0C9474
:1006400000000F931F93CF93DF930E941213823009
:1006500019F40EE412E002C004EF11E082E00E94FF
:100660003D06EC010E942E139C0180917E0188239F
:1006700019F481E080937E0180917E019927813079
:10068000910531F0813091054CF104973CF50EC095
:1006900005501040C017D1070CF582E080937E0111
:1006A00064962C173D07D4F483E016C0CE014E9615
:1006B000821793071CF482E080937E01CE0144965A
:1006C000281739071CF483E080937E010B5F1F4FCE
:1006D0000C171D071CF481E080937E0180917E0140
:1006E00090917E00823021F4903229F0DD9A03C08F
:1006F000903209F0DD98DF91CF911F910F9108950D
:100700000F931F9380917F0199278130910559F1B3
:10071000823091051CF4892B89F045C0029709F0BD
:1007200042C080918A0090918B00019790938B003A
:1007300080938A00892B11F410927F0185E00E943A
:100740003D068B5892405CF485E00E943D068C018A
:1007500084E00E943D06C2968017910724F581E04F
:1007600080937F0120C085E00E943D068C0186E0D9
:100770000E943D06081B190B0E311105A4F485E0FB
:100780000E943D068C0184E00E943D06C296081737
:1007900019074CF482E080937F0180EE91E0909302
:1007A0008B0080938A0080917F0190917E00813040
:1007B00021F4903229F0DE9A03C0903209F0DE98DD
:1007C0000E9464121F910F910895CF93DF93CDB7CC
:1007D000DEB728970FB6F894DEBF0FBECDBF88E016
:1007E000A0E6B0E0FE0131960D9001928A95E1F706
:1007F000409187012091880130918901542F5270D6
:1008000041FDF3C0C9014897059710F4477F0AC01E
:10081000225330402530310510F4486003C0509316
:100820008C0044604093870140918201842F855160
:100830008730E0F4FE017497E40FF11D30918701D9
:10084000232F26952695269521708081829F902DB5
:10085000112480918101890F80938101932F9170E0
:100860009227832F8E7F892B80938701842F8D5130
:100870008630E0F4FE017C97E40FF11D3091870192
:10088000232F26952695269521708081829F902D75
:10089000112480918001890F80938001932F9170A2
:1008A0009227832F8E7F892B80938701842F8452F8
:1008B0008630E0F4FE01B397E40FF11D309187011B
:1008C000232F26952695269521708081829F902D35
:1008D000112480918301890F80938301932F91705C
:1008E0009227832F8E7F892B80938701842F8A52B2
:1008F0008330E0F4FE01B997E40FF11D30918701D8
:10090000232F26952695269521708081829F902DF4
:10091000112480918401890F80938401932F917019
:100920009227832F8E7F892B80938701842F8D526E
:100930008530E0F4FE01BC97E40FF11D3091870192
:10094000232F26952695269521708081829F902DB4
:10095000112480918501890F80938501932F9170D7
:100960009227832F8E7F892B80938701842F825338
:100970008830E0F4FE01F197E40FF11D309187011A
:10098000232F26952695269521708081829F902D74
:10099000112480918601890F80938601932F917095
:1009A0009227832F8E7F892B809387014C3121F0F2
:1009B000433211F04A33A9F420918701822F8695A2
:1009C000869586958170922F9170891729F0246001
:1009D0002093870110928C00809187018E7F8093F5
:1009E00087014F5F4093820139C0235C3140B0F1F1
:1009F000809182018B3309F5942F947042FD1DC0C4
:100A00008091800180938A018091810180938B0184
:100A100090938C0180918601809390018091850153
:100A200080938F018091830180938D018091840157
:100A300080938E0181E080938C004A7F40938701F0
:100A40001092800110928101109282011092830114
:100A500010928501109286011092840128960FB69B
:100A6000F894DEBF0FBECDBFDF91CF91089580B364
:100A700086958695282F33272170307050918701F5
:100A8000452F46954170842F99272817390779F00B
:100A900040954170440F852F8D7F842B8093870173
:100AA0000E94E503109289011092880109C080918B
:100AB0008801909189010196909389018093880122
:100AC00090918D00915090938D009923D9F480914D
:100AD0008C018F5F80938C018C33A0F090938C01FC
:100AE00080918B018F5F80938B018C3358F09093B2
:100AF0008B0180918A018F5F80938A01883110F089
:100B000090938A010895E62FFF27EE0FFF1FE80F4D
:100B1000F91F859194910E940E0B0895FF920F93F7
:100B20001F93CF93DF93CDB7DEB727970FB6F89417
:100B3000DEBF0FBECDBFF62EAA2797FDA095BA2F18
:100B4000BC01CD010E945D17DC01CB0120E030E04B
:100B500040E251E4BC01CD010E946916DC01CB01E9
:100B60008E010F5F1F4F21E0422FBC01CD010E947B
:100B7000AF16CE0101960E94000BFF2019F08F2DB9
:100B80000E94E10A27960FB6F894DEBF0FBECDBFD4
:100B9000DF91CF911F910F91FF9008951F93CF93F5
:100BA000DF93CDB7DEB727970FB6F894DEBF0FBE41
:100BB000CDBF162F4AE050E0BE016F5F7F4F0E940D
:100BC000C615CE0101960E94000B112319F0812F4A
:100BD0000E94E10A27960FB6F894DEBF0FBECDBF84
:100BE000DF91CF911F91089560E083E10E94CC0ACC
:100BF00080918A018A3018F480E20E94E10A809193
:100C00008A016AE399270E94CE0580918B018A3080
:100C100018F480E30E94E10A80918B016AE399272E
:100C20000E94CE0580918C018A3018F480E30E94E6
:100C3000E10A80918C0160E099270E94CE05089519
:100C4000CF93C82F883218F480E20E94E10A8C2FDB
:100C5000869586956AE399270E94CE058C2F83702E
:100C600019F480E30E94E10A60E08FE0C89FC001B0
:100C700011240E94CE05CF91089591E090939101A7
:100C8000E82FFF27EE0FFF1FE057FF4F8081918174
:100C900010929101089580918E008F5F80938E0055
:100CA000803110F010928E0080918E00883010F408
:100CB00086E101C088E180936A0008951F920F9237
:100CC0000FB60F9211242F933F934F935F936F931F
:100CD0007F938F939F93AF93BF93EF93FF9381B1D4
:100CE000887F8093920180919201992788329105A3
:100CF00069F18932910584F480319105F1F08131F7
:100D000091051CF40897C9F04AC088319105C1F0DB
:100D1000809709F440C043C088349105E1F18934DB
:100D2000910524F480349105B9F039C080359105DE
:100D3000A9F088359105B1F032C080916A0003C0F6
:100D400080918E00877083B985E82BC080916A00FE
:100D50008F5F80936A0021C085EC23C083B18093AC
:100D60008F00F2CF81E08093910180918E00E82F77
:100D7000FF27EE0FFF1FE057FF4F80918F00282FB6
:100D8000332783B19927982F8827282B392B208345
:100D90003183109291010E944B0685EA02C016BE73
:100DA00007C086BF80E095E090936900809368005B
:100DB000FF91EF91BF91AF919F918F917F916F9133
:100DC0005F914F913F912F910F900FBE0F901F9009
:100DD000189584E680B983E081B985EA86BF80E012
:100DE00095E0909369008093680008958091970141
:100DF00090919801A0919901B0919A01BC01CD0107
:100E000024E630E040E050E00E944D19DC01CB01C7
:100E1000BC01CD0120E037E740E050E00E948B1993
:100E2000DA01C901992708952F923F924F925F925C
:100E30006F927F928F929F92AF92BF92CF92DF92EA
:100E4000EF92FF920F931F93CF93DF93CDB7DEB74F
:100E500060970FB6F894DEBF0FBECDBF80919601AC
:100E600099278130910519F0029721F006C087E09B
:100E700090E007C088E090E004C087E00E943D0653
:100E800014C10E94B3159927AA2797FDA095BA2FE0
:100E9000BC01CD010E945D17DC01CB0120E030E0F8
:100EA00040E251E4BC01CD010E94691669837A8356
:100EB0008B839C838BE00E943D06AA2797FDA0951B
:100EC000BA2FBC01CD010E945D17DC01CB0120E0EF
:100ED00030E040E251E4BC01CD010E9469166D830F
:100EE0007E838F8398878AE090E00E94B315182F45
:100EF000992787FD9095A92FB92FBC01CD010E949C
:100F00005D176B017C0117FF08C020E030E040E86E
:100F100053E40E941F166B017C018BE090E00E945D
:100F2000B3159927AA2797FDA095BA2FBC01CD012B
:100F30000E945D17DC01CB0120E030E040E251E48B
:100F4000BC01CD010E94691669877A878B879C87CF
:100F500086E090E00E94B3159927AA2797FDA095F7
:100F6000BA2FBC01CD010E945D17DC01CB0120E04E
:100F700030E040E251E4BC01CD010E9469166D876A
:100F80007E878F87988B89E090E00E94B315992720
:100F900087FD9095A92FB92FBC01CD010E945D1747
:100FA0001B012C019B01AC016D817E818F81988595
:100FB0000E946717882324F42D823E824F82588630
:100FC00029813A814B815C816D817E818F819885F9
:100FD0000E946A1788232CF069817A818B819C8119
:100FE00056C029813A814B815C81C701B6010E94BC
:100FF0001E163B014C0129853A854B855C8560E0D6
:1010000070E080E89FE30E9469165B016C012D810E
:101010003E814F81588569817A818B819C810E94B4
:101020001E167B018C01A201910169817A818B815D
:101030009C810E941E16DC01CB019C01AD01C80100
:10104000B7010E946916DC01CB01A6019501BC0124
:10105000CD010E942918DC01CB019C01AD01C40126
:10106000B3010E94DB17DC01CB019C01AD0169815A
:101070007A818B819C810E941F16DC01CB012D851A
:101080003E854F855889BC01CD010E941F1620E086
:1010900030E040E251E40E94DB17DC01CB01BC01EF
:1010A000CD010E944017DC01CB0160960FB6F89489
:1010B000DEBF0FBECDBFDF91CF911F910F91FF908B
:1010C000EF90DF90CF90BF90AF909F908F907F90E8
:1010D0006F905F904F903F902F9008950F931F93C4
:1010E00080916B0099278130910509F49BC0823073
:1010F00091051CF4892B49F0CBC08230910509F48D
:10110000A2C0039709F4B9C0C3C00E9414078C01A0
:1011100087E00E943D06F801E81BF90B86E490E0A9
:10112000E89FB001E99F700DF89F700D1124809128
:101130009301909194019F01281B390B8CE390E05F
:10114000289FA001299F500D389F500D1124640F36
:10115000751F77FF03C0709561957F4F61387105EA
:1011600008F455C09B014427552780919701909121
:101170009801A0919901B0919A011E161F061CF5C5
:10118000820F931FA41FB51F80939701909398011E
:10119000A0939901B0939A0181509747A040B04025
:1011A00064F080E097E7A0E0B0E08093970190932F
:1011B0009801A0939901B0939A0180917E008032AA
:1011C000E9F0DA9A1BC0821B930BA40BB50B80933A
:1011D000970190939801A0939901B0939A01B7FF5A
:1011E00008C01092970110929801109299011092E4
:1011F0009A0180917E00803209F0DA9881E0809334
:101200006B0080917E00803221F0DB9A02C060E0AA
:1012100078E2F0939401E093930170936D006093F2
:101220006C0036C080917E00803209F0DB988032FD
:1012300009F0DA9880E09EE190936D0080936C0055
:1012400010926B0025C080917E00803209F0DA9800
:10125000803209F0DB9A83E080936B0080E098E7AE
:1012600090936D0080936C001092970110929801FA
:101270001092990110929A010BC080917E008032E9
:1012800009F0DB9880E09EE190936D0080936C0004
:101290001F910F9108950F931F93CF93DF9383E0D6
:1012A00090E00E94B315C82FDD27C230D105E9F1C7
:1012B000C330D1053CF4209709F43EC0C130D105BC
:1012C00039F03AC0C330D10581F1249791F134C08F
:1012D00000918A01000F000F80918B016FE00E9446
:1012E0006C19080F84E090E00E94B315182F85E078
:1012F00090E00E94B315811738F084E090E00E94DE
:10130000B315081778F006C084E090E00E94B3158A
:10131000081730F485E090E00E94B315081710F428
:10132000CE0104C080E090E001C082E0809396018D
:1013300005C081E080939601109296018BE00E9497
:101340003D068C0181E090E00E94B3159927039639
:10135000081719071CF082E0809395018BE00E942A
:101360003D068C0182E090E00E94B3159927039618
:101370008017910784F48BE00E943D068C0181E088
:1013800090E00E94B31599270397081719071CF4DA
:1013900081E0809395018BE00E943D068C0182E004
:1013A00090E00E94B315992703970817190714F4C2
:1013B0001092950180919601813031F480919501D0
:1013C000823011F41092960180919601823031F4AE
:1013D00080919501882311F01092960180919601D9
:1013E000882329F080919B01882319F482E080935F
:1013F0009B0180919B0199278230910519F00397F9
:10140000B9F023C00E941213882331F40E942E13D6
:101410008B539140D4F40AC00E942E138C010A50C1
:1014200010400E941407081719077CF483E00BC0D2
:101430000E942E138C010E5110400E941407801739
:1014400091071CF482E080939B0180919B01909115
:101450007E00823051F4903209F0DF9A80916B0067
:10146000823078F010926B000AC0903209F0DF9859
:1014700080916B00823028F482E080936B000E94A0
:101480006E08DF91CF911F910F91089521E030E018
:1014900000909C0102C0220F331F0A94E2F782B32E
:1014A000822B82BB00C0922F909582B3892382BB8E
:1014B00008950F931F93082F662311F0959A01C08A
:1014C0009598949884B38C6384BB25B3237C1127AF
:1014D000C801807F90709595879595958795282B65
:1014E00025BB0E94460A85B3837C0F701070000FE5
:1014F000111F000F111F802B85BB0E94460A85B368
:101500008C6385BB1F910F910895882311F0959AE4
:1015100001C09598949A84B3837C84BB21E030E029
:1015200000909C0102C0220F331F0A94E2F782B39D
:10153000822B82BB00C093B3990F990F907F422FEB
:10154000409582B3842382BB00C082B3822B82BBCE
:1015500000C083B3869586958F70982B82B38423C1
:1015600082BB892F9927089580E00E94850A8823ED
:10157000DCF383E090E00197F1F780E00E94850AB8
:10158000992708951F93182F0E94B40A60E0812FB5
:101590000E94590A1F910895982F623028F087E021
:1015A00080939C01625003C086E080939C01629509
:1015B000660F660F607C690F862F80580E94C20AF2
:1015C0000895CF93C82F0E94B40ACA3099F48B3182
:1015D00010F490E40AC090E080919C01863011F4F0
:1015E00087E001C086E080939C01892F80580E948B
:1015F000C20A04C061E08C2F0E94590ACF9108955D
:10160000CF93DF93EC018991882329F00E94E10AAE
:1016100089918823D9F7DF91CF910895CF93DF93F4
:10162000EC01FC0121968491882339F00E94E10AA3
:10163000FE01219684918823C9F7DF91CF91089507
:1016400087E080939C0181E00E94C20A86E080933B
:101650009C0181E00E94C20A08951F93182F85B350
:10166000837C8C6085BB0E94460A80EF93E20197E1
:10167000F1F70E94460A85E790E00197F1F70E9492
:10168000460A85E790E00197F1F785B3837C88608F
:1016900085BB0E94460A85E790E00197F1F788E252
:1016A0000E94C20A88E00E94C20A81E00E94C20A27
:1016B00086E00E94C20A812F0E94C20A1F910895EB
:1016C0001F93182F84B38C6384BB8D9A8C9A8E9A47
:1016D0008F9A80E393E70197F1F787E080939C016D
:1016E000812F0E942D0B86E080939C01812F0E9408
:1016F0002D0B1F91089580919E01815080939E0132
:101700008823D1F480919F01282F332786B399270E
:10171000807F90702817390761F086B3807F8093AF
:101720009F01803F11F080939D018AE080939E018C
:10173000089581E080939E01089580919D0110920B
:101740009D019927803B910599F0813B910524F4F7
:101750008037910581F012C0803D910531F0803EC7
:10176000910561F481E090E0089582E090E00895B1
:1017700083E090E0089584E090E0089580E090E0B8
:1017800008951F93CF93DF9310BC8FE289B988E04F
:101790008AB986E880BD8CE00E94600B8CE294E000
:1017A0000E940E0B80E40E94C20ACEE6D0E01FE049
:1017B000FE01849161E070E099270E94590A11505E
:1017C000219617FFF5CF62E080E00E94CC0A80E40A
:1017D0000E94C20ACEE6D0E01FE0FE01849161E0E3
:1017E00070E099270E94590A1150219617FFF5CFF2
:1017F00078948FEF8ABB84B3806C84BB17BAC39A8A
:1018000088B3806F88BB0E94E90680EC98EA9BBD94
:101810008ABD85E08EBD08B604FEFDCF88B7806125
:1018200088BF1EBC8FE790E79BBD8ABD89E08EBD57
:1018300080E189BFDF91CF911F910895CFE5D4E07A
:10184000DEBFCDBF0E94C10BC0E00E949D0B88236C
:1018500011F00E94F41180918C01C81729F080E1E9
:101860000E94F411C0918C018091A00180FF05C0FD
:101870008E7F8093A0010E94F3128091A00181FFCE
:1018800005C08D7F8093A0010E946E088091A00109
:1018900083FF05C0877F8093A0010E944113909130
:1018A000A00194FFD2CF80918C00882371F29F7E9B
:1018B0009093A0010E94F514C8CF81E080937F012E
:1018C0000E948003089508958EE295E00E940E0B19
:1018D0000E94F40561E08FE00E94CC0A60917E01D5
:1018E00085EF92E00E94830562E08AE00E94CC0AC4
:1018F00060919B018DEF92E00E94830563E089E097
:101900000E94CC0A0E941213682F8FEE92E00E9470
:10191000830580E20E94E10A0E942E136FED0E946F
:101920008E0508950F931F9382E895E00E940E0B99
:101930000E94F40561E08CE00E94CC0A85E00E94E0
:101940003D066FED0E948E0561E084E10E94CC0AA5
:1019500084E00E943D066FED0E948E0562E08CE0FF
:101960000E94CC0A86E00E943D066FED0E948E0523
:1019700062E084E10E94CC0A83E00E943D066FEDA4
:101980000E948E0563E089E00E94CC0A60917F018D
:101990008DE093E00E94830580917F01992781303B
:1019A000910519F0029779F015C085E00E943D0677
:1019B0008C0186E00E943D066FED081B190BC801E3
:1019C0000E948E0507C060E080918A0090918B0094
:1019D0000E94CE051F910F91089583EE95E00E941D
:1019E0000E0B0E94F40561E088E00E94CC0A82E0C0
:1019F0000E943D066FED0E948E0561E08EE00E9420
:101A0000CC0A60917E0185EF92E00E94830562E03E
:101A100088E00E94CC0A81E00E943D066FED0E94A2
:101A20008E0563E088E00E94CC0A80E00E943D06BB
:101A30006FED0E948E0508958EEA95E00E940E0BD0
:101A40000E94F40561E08CE00E94CC0A87E00E94CD
:101A50003D066FED0E948E0562E08CE00E94CC0A8C
:101A600088E00E943D066FED0E948E0562E083E1F2
:101A70000E94CC0A0E94F60665E299270E94CE05D4
:101A800063E087E00E94CC0A0E9414076FED0E9479
:101A90008E0563E085E10E94CC0A8BE00E943D0642
:101AA0006FED0E948E0561E083E10E94CC0A609197
:101AB0009B018DEF92E00E948305089587E595E0F4
:101AC0000E940E0B0E94F40561E08CE00E94CC0A9B
:101AD00089E00E943D066FED0E948E0562E08CE079
:101AE0000E94CC0A8AE00E943D066FED0E948E059E
:101AF00063E089E00E94CC0A6091B60085E093E043
:101B00000E948305089581E295E00E940E0B0895DE
:101B10008BE794E00E940E0B61E08FE00E94CC0AFC
:101B20008CE00E94C20A82EA91E00E94B315682FFD
:101B300086EB92E00E94830562E087E00E94CC0A77
:101B40008CE090E00E94B3150E94200663E087E0DD
:101B50000E94CC0A8DE090E00E94B3150E942006FE
:101B600008958DE994E00E940E0B61E08FE00E94E1
:101B7000CC0A8CE00E94C20A83E090E00E94B31578
:101B8000682F8CEA92E00E94830562E087E00E9461
:101B9000CC0A84E090E00E94B3150E94200663E026
:101BA00087E00E94CC0A85E090E00E94B3150E9475
:101BB000200608958FEE94E00E940E0B61E08FE006
:101BC0000E94CC0A8CE00E94C20A8BE090E00E9446
:101BD000B31560E099270E948E0562E08FE00E94B5
:101BE000CC0A8AE090E00E94B3156FED99270E941D
:101BF000CE0563E08FE00E94CC0A8CE00E94C20A0E
:101C000089E090E00E94B3156FED992787FD9095CC
:101C10000E94CE0508958BEB94E00E940E0B61E0CC
:101C20008EE00E94CC0A8CE00E94C20A87E090E01D
:101C30000E94B3156FED99270E948E0562E08EE039
:101C40000E94CC0A88E090E00E94B3156FED9927BE
:101C50000E948E0563E08EE00E94CC0A8CE00E9418
:101C6000C20A86E090E00E94B3156FED992787FDC8
:101C700090950E948E05089584E594E00E940E0BD5
:101C800061E08EE00E94CC0A8CE00E94C20A81E0F2
:101C900090E00E94B31560E099270E948E0562E0F3
:101CA0008EE00E94CC0A82E090E00E94B31560E0D2
:101CB00099270E948E05089580E494E00E940E0BFF
:101CC00061E082E00E94CC0A8CE00E94C20A80E0BF
:101CD00090E00E94B3156FED99270E94CE050895FC
:101CE0008091B0009091B10001969093B1008093E3
:101CF000B0002091B4003091B5002817390724F4C2
:101D00003093B1002093B00008958091B00090917D
:101D1000B10001979093B1008093B0002091B20080
:101D20003091B3008217930724F43093B1002093CD
:101D3000B00008952091B0003091B1004091B400FE
:101D40005091B500421753073CF08091B20090913A
:101D5000B300281739078CF42091B2003091B300FA
:101D6000CA01821B930B97FD019695958795280FC5
:101D7000391F3093B1002093B00008950E94830D65
:101D800061E0862F0E94CC0A6091B0008BED92E05A
:101D90000E948305089586E090E09093B1008093BF
:101DA000B0001092B3001092B20089E090E09093DE
:101DB000B5008093B4000E94BE0E08950E94700E7C
:101DC0000E94BE0E08950E94850E0E94BE0E0895C8
:101DD000CF938091B0009091B1008830910564F468
:101DE00021E030E002C0220F331F8A95E2F78BB367
:101DF00082278BBBCBB30CC0029721E030E002C03E
:101E0000220F331F8A95E2F785B3822785BBC5B3BE
:101E1000C2230E94BE0ECC2319F086E094E002C0DB
:101E20008EE194E00E940E0BCF91089561E08FE067
:101E30000E94CC0A6091B00086EB92E00E9483057C
:101E400008950E94880D82EA91E00E94B3159927B7
:101E50009093B1008093B0001092B3001092B20042
:101E600083E090E09093B5008093B4000E949A0EB6
:101E70000E94160F8FE00E94C20A08950E94700E01
:101E80000E94160F08950E94850E0E94160F089555
:101E900062E087E00E94CC0A8091B0000E94200698
:101EA00008956091B00082EA91E00E94BB150E9403
:101EB000880D8CE090E00E94B31599279093B100B3
:101EC0008093B0001092B3001092B2008FE590E0C2
:101ED0009093B5008093B4000E949A0E0E94480F20
:101EE0008FE00E94C20A08950E94700E0E94480F5F
:101EF00008950E94850E0E94480F089563E087E0D0
:101F00000E94CC0A8091B0000E9420060895609142
:101F1000B0008CE090E00E94BB150E94880D8DE01F
:101F200090E00E94B31599279093B1008093B00080
:101F30001092B3001092B2008FE590E09093B5003C
:101F40008093B4000E949A0E0E947E0F8FE00E9440
:101F5000C20A08950E94700E0E947E0F08950E948A
:101F6000850E0E947E0F08956091B0008DE090E094
:101F70000E94BB150E94210F089561E08FE00E942E
:101F8000CC0A6091B0008CEA92E00E94830508952B
:101F90000E94B10D83E090E00E94B31599279093C1
:101FA000B1008093B0001092B3001092B20084E0B0
:101FB00090E09093B5008093B4000E949A0E0E9426
:101FC000BD0F8FE00E94C20A08950E94700E0E9409
:101FD000BD0F08950E94850E0E94BD0F089562E016
:101FE00087E00E94CC0A8091B0000E9420060895EC
:101FF0006091B00083E090E00E94BB150E94B10D9B
:1020000084E090E00E94B31599279093B1008093EB
:10201000B0001092B3001092B2008FE590E0909360
:10202000B5008093B4000E949A0E0E94EF0F8FE0DB
:102030000E94C20A08950E94700E0E94EF0F089538
:102040000E94850E0E94EF0F089563E087E00E94D2
:10205000CC0A8091B0000E94200608956091B000E3
:1020600084E090E00E94BB150E94B10D85E090E0F5
:102070000E94B31599279093B1008093B0000E94FD
:102080009A0E0E9425108FE00E94C20A08950E94B5
:10209000700E0E94251008950E94850E0E94251042
:1020A00008956091B00085E090E00E94BB150E9409
:1020B000C80F089561E08FE00E94CC0A60E0809133
:1020C000B0009091B1000E948E0508950E94DA0D33
:1020D0008BE090E00E94B31599279093B100809314
:1020E000B00081E090E09093B3008093B2008EE165
:1020F00090E09093B5008093B4000E949A0E0E94E5
:102100005A108FE00E94C20A08950E94700E0E9429
:102110005A1008950E94850E0E945A10089562E098
:102120008FE00E94CC0A6FED8091B0009091B100D9
:102130000E94CE0508956091B0008BE090E00E946F
:10214000BB150E94DA0D8AE090E00E94B315992732
:102150009093B1008093B00083E290E09093B3003D
:102160008093B2008CE390E09093B5008093B4002C
:102170000E949A0E0E948F108FE00E94C20A08955A
:102180000E94700E0E948F1008950E94850E0E947A
:102190008F10089563E08FE00E94CC0A6FED80916C
:1021A000B0009091B1000E94CE0508956091B000FA
:1021B0008AE090E00E94BB150E94DA0D89E090E071
:1021C0000E94B315992787FD90959093B100809355
:1021D000B00081EF9FEF9093B3008093B200109214
:1021E000B5001092B4000E949A0E0E94CA108FE0AF
:1021F0000E94C20A08950E94700E0E94CA1008959B
:102200000E94850E0E94CA1008956091B00089E076
:1022100090E00E94BB150E946610089561E08EE078
:102220000E94CC0A60E08091B0009091B1000E94C1
:102230008E0508950E940B0E87E090E00E94B31572
:1022400099279093B1008093B00080EA90E090933A
:10225000B3008093B2008FEF90E09093B50080932D
:10226000B4000E949A0E0E940E118FE00E94C20AD2
:1022700008950E94700E0E940E1108950E94850E0E
:102280000E940E11089562E08EE00E94CC0A60E088
:102290008091B0009091B1000E948E0508956091E8
:1022A000B00087E090E00E94BB150E940B0E88E012
:1022B00090E00E94B31599279093B1008093B000ED
:1022C0000E949A0E0E9443118FE00E94C20A089554
:1022D0000E94700E0E94431108950E94850E0E9474
:1022E0004311089563E08EE00E94CC0A60E0809183
:1022F000B0009091B1000E948E0508956091B000E9
:1023000088E090E00E94BB150E940B0E86E090E0F2
:102310000E94B31599279093B1008093B0008DE986
:102320009FEF9093B3008093B20083E690E0909388
:10233000B5008093B4000E949A0E0E9472118FE043
:102340000E94C20A08950E94700E0E9472110895A0
:102350000E94850E0E94721108956091B00086E07F
:1023600090E00E94BB150E941A11089561E082E07E
:102370000E94CC0A6FED8091B0009091B1000E9454
:10238000CE0508950E945C0E80E090E00E94B31597
:1023900099279093B1008093B00089E190E09093E9
:1023A000B3008093B2008CE390E09093B5008093EB
:1023B000B4000E949A0E0E94B6118FE00E94C20AD9
:1023C00008950E94700E0E94B61108950E94850E15
:1023D0000E94B61108956091B00080E090E00E94E4
:1023E000BB150E945C0E08950F931F93CF93DF934C
:1023F000CDB7DEB725970FB6F894DEBF0FBECDBFC1
:10240000082F10E085E0189FC00111248C559F4FC4
:102410001F5F45E050E0BC01CE0101960E94EB1524
:102420009981992339F08A81801761F780917E0024
:10243000981741F7992359F08D818F3F29F00E9419
:10244000200B8D8180937E00EB81FC810995259680
:102450000FB6F894DEBF0FBECDBFDF91CF911F91B5
:102460000F9108951F93CF93C0918A01CC0FCC0F89
:1024700080918B016FE00E946C19C80F8CE090E096
:102480000E94B315182F8DE090E00E94B3158117BC
:1024900038F08CE090E00E94B315C81780F006C0B9
:1024A0008CE090E00E94B315C81730F48DE090E006
:1024B0000E94B315C81718F481E090E002C080E0D4
:1024C00090E0CF911F910895CF93C0E082EA91E010
:1024D0000E94B315982F8091B600882311F08330A5
:1024E00021F580917F01882309F04AC080919B01EA
:1024F000833029F4892F8250823008F4C1E0809122
:102500007E01833029F4913011F0933009F4C1E059
:102510000E9432128823A1F1CC2391F180917E0098
:10252000803209F0AE9A81E026C080917E01813030
:1025300021F0892F8250823008F0CFEF80919B01EB
:10254000882321F0913019F0933009F0C150809127
:102550007F018111CEEF0E943212882311F0CE3F0D
:1025600079F480917E00803209F0AE988091B600B7
:10257000823021F483E08093B60002C01092B6004E
:102580008091B60099278130910549F082309105FC
:102590001CF4892B09F125C0029781F022C089E043
:1025A0000E943D06855A9140E4F082E08093B60097
:1025B00080917E008032A9F0D99A13C089E00E94F0
:1025C0003D06805991406CF481E08093B600809183
:1025D0007E00803231F004C080917E00803209F0AC
:1025E000D998CF9108950F931F9380E00E943D06E4
:1025F0008C0181E00E943D069801281B390B203593
:1026000031052CF080917E00803209F0DC9A29326D
:1026100031052CF480917E00803209F0DC981F9106
:102620000F9108958091B60099278130910531F07E
:10263000813091054CF004973CF403C080E090E0B9
:10264000089581E090E0089580917F01813019F430
:1026500082E090E0089580E090E008950E941213D7
:1026600099278130910519F0029719F006C089E089
:1026700001C085E00E943D06089584E00E943D0669
:102680000895CF93DF930E94800380E090E00E9442
:10269000B3159AE0899FE00111240E9421038091E3
:1026A0007E01823031F0833089F40E941213882336
:1026B00069F082E00E943D0625978C179D0730F453
:1026C00080919B01823049F481E005C080919B019B
:1026D000813019F482E080939B010E944B090E9493
:1026E0006412DF91CF9108951F920F920FB60F924F
:1026F00011242F933F934F935F936F937F938F9307
:102700009F93AF93BF93EF93FF930E9437050E946F
:102710007B0BB4990AC081E08093A10188EE93E01D
:1027200090938800809387000DC0809187009091DE
:10273000880001979093880080938700892B11F47B
:102740001092A1018091850090918600019790934D
:10275000860080938500892B59F480E09CE3909358
:102760008600809385008091A00181608093A00104
:1027700080916C0090916D00019790936D00809313
:102780006C00892B59F488EE93E090936D00809350
:102790006C008091A00182608093A00180918300F1
:1027A0009091840001979093840080938300892BFB
:1027B00059F480E09EE1909384008093830080919F
:1027C000A00188608093A00180917F00909180009B
:1027D000A0918100B09182000197A109B109809375
:1027E0007F0090938000A0938100B09382000097B7
:1027F000A105B10589F480E09AE0A0E0B0E0809303
:102800007F0090938000A0938100B093820080911C
:10281000A00180618093A00180916800909169007F
:10282000019790936900809368008091680090916F
:102830006900892B11F40E94E906FF91EF91BF9185
:10284000AF919F918F917F916F915F914F913F9148
:102850002F910F900FBE0F901F9018951F920F92FF
:102860000FB60F9211248F939F93EF93FF93809154
:10287000B90081508093B9008F3F79F08091B70003
:102880009091B800FC01E654FF4F01969093B80078
:102890008093B70080818CB901C05598FF91EF916A
:1028A0009F918F910F900FBE0F901F901895CF930F
:1028B000DF93EC01862F9927009721F0019709F407
:1028C00040C05AC08091B900282F332726543F4F6B
:1028D000CE016AE070E00E947819CB014AE050E036
:1028E000B9010E94C6158091B900A82FBB27A65434
:1028F000BF4FFD0101900020E9F731979E2F9A1BF1
:10290000980FE92FFF27E654FF4F8EE28083892F2F
:102910008F5F282F332726543F4F8F5F8093B90056
:10292000CE01D7FF04C0882799278C1B9D0B6AE036
:1029300070E00E9478194AE050E0B9010E94041644
:102940001BC08091B900992786549F4F4AE050E000
:10295000BC01CE010E9404168091B900A82FBB27AC
:10296000A654BF4FFD0101900020E9F73197EA1B03
:10297000FB0B8E0F8093B9008091B900E82FFF27E1
:10298000E654FF4F9BE390838F5F8093B900DF9104
:10299000CF910895282F8A3058F48091B900E82FFC
:1029A000FF27E654FF4F90E390838F5F8093B90039
:1029B0008091B900992786549F4F4AE050E0BC01AE
:1029C000822F99270E9404168091B900A82FBB2757
:1029D000A654BF4FFD0101900020E9F73197EA1B93
:1029E000FB0B8E0F8093B90008951F938BE18093AA
:1029F000BA0080E18093BB0082E08093B9008091AF
:102A00008D010E94CA148091B900E82FFF27E65477
:102A1000FF4F1EE210838F5F8093B90080918F017A
:102A20000E94CA148091B900E82FFF27E654FF4F97
:102A300010838F5F8093B900809190010E94CA1427
:102A40009091B900E92FFF27E654FF4F80E2808381
:102A50009F5F9093B90080918A010E94CA1480916F
:102A6000B900E82FFF27E654FF4F1AE310838F5F6A
:102A70008093B90080918B010E94CA148091B900A3
:102A8000E82FFF27E654FF4F10838F5F8093B90034
:102A900080918C010E94CA149091B900E92FFF2700
:102AA000E654FF4F8BE380839F5F9093B900809142
:102AB0008E0161E099270E94571410E0812F0E9437
:102AC0003D0660E00E9457141F5F1C30B8F30E945F
:102AD000140760E00E9457148BB3282F332785B367
:102AE0009927807C9070880F991F880F991F61E04B
:102AF000822B932B0E94571480917E0161E09927CD
:102B00000E94571480919B0161E099270E945714FD
:102B100080917F0161E099270E9457148091B6004F
:102B200061E099270E9457140E94F60661E09927F8
:102B30000E9457148091B900E82FFF27E654FF4FF9
:102B40009BE190838F5FE82FFF27E654FF4F91E1D1
:102B500090838F5F8093B9001092B8001092B700F5
:102B6000559A1F910895E199FECF9FBB8EBBE09AC5
:102B700099278DB30895E199FECF9FBB8EBB6DBBA6
:102B80000FB6F894E29AE19A0FBE0895E62FF72F58
:102B90002E2F3F2FE8944230CCF04532BCF44A301F
:102BA00029F497FB1EF4909581959F4F642F77270A
:102BB0000E94A619805D8A330CF0895D8193862F6F
:102BC000972F009799F716F45DE25193932F822F78
:102BD00010820C94F415FB01DC0102C005900D92EB
:102BE00041505040D8F70895DC01FC0101900020CD
:102BF000E9F73297AE17BF0730F47C91608170839C
:102C000031976D93F7CF0895E62FF72F2E2F3F2F93
:102C100042307CF045326CF4642F77270E94A6196D
:102C2000805D8A330CF0895D8193862F972F009702
:102C300099F7932F822F10820C94F4155058192E67
:102C400088D101D06BC1BA17620773078407950753
:102C5000B1F188F40EF410940B2EBA2FA02D062E8D
:102C6000622F202D072E732F302D082E842F402DFC
:102C7000092E952F502DFF275523B9F0591B49F0E8
:102C8000573E98F0469537952795A795F040539570
:102C9000C9F776F0BA0F621F731F841F30F487954F
:102CA00077956795B795F040939517FA0F2E08958D
:102CB000BF1BBB27BA0B620B730B840BF6CFDEF680
:102CC00065C1592F482F372F262F9FE380E877279C
:102CD00066273FD101D022C1552359F0992369F0CD
:102CE0009F575F57951B33F442F4903811F4915875
:102CF00005C02CC191589F3F09F448C1BB2711243E
:102D000062177307840730F4660F771F881FBB1F95
:102D1000915098F311D00F920FD00F920DD0A0E8E0
:102D20002617370748071B0609F0A048BA2F602D61
:102D30007F918F9100240895A0E800246217730703
:102D40008407B10528F0621B730B840BB1090A2AB2
:102D5000660F771F881FBB1FA69581F70895DF9325
:102D6000CF931F930F93E8018C01000F111F1F3F9A
:102D700031F49EE481E49993899399937AC04F93B7
:102D800099231AF40DE209939F77022F03959F93DD
:102D90008F937F936F93622F7727882799270E94BD
:102DA0005D179068AC019B0191E480E2772766276C
:102DB0000E9429185FEF4FEF0E94C8172F913F9193
:102DC0004F915F910E941F16102F013009F40027C8
:102DD00051E440E2332722276217730784079507DF
:102DE00024F00E9469161395F3CF9F938F937F93DE
:102DF0006F930E944017562F505D59930E945D17A4
:102E00002F913F914F915F910E941E16905851E46F
:102E100040E2332722270E94DB17101711F45EE2ED
:102E200059931A9511F718825F91EF91FF91FF93D3
:102E3000EF93452F442312F440954395CE01BF01F3
:102E4000861B970B142F181B90E284179CF45523B4
:102E50006AF021963196E40FF11D83955A915293B1
:102E60008A95E1F792931A95E9F704C099931A9518
:102E7000E9F718828F919F918C01CF91DF9108958E
:102E800097FB73D09F3738F0FEE9F91B982F872FF7
:102E9000762F6B2F05C077C09695879577956795A8
:102EA000F150D0F73EF490958095709561957F4FE5
:102EB0008F4F9F4F0895E89403C097FB0EF4F3DF04
:102EC000B62F672F782F892F9EE9002427C00ED0B8
:102ED0005EF004C00BD026F001C008D019F020F439
:102EE0008FEF089580E0089581E0089597FB092E03
:102EF000052600F8689430D0E89407FC07C06217F4
:102F000073078407950721F008F4009407949894B8
:102F100008959A95BB0F661F771F881F1124992368
:102F2000A1F08823B2F79F3F59F0BB0F48F421F47A
:102F3000002011F460FF04C06F5F7F4F8F4F9F4FE1
:102F4000881F9795879597F908951DC09FEF80EC8E
:102F50000895052E092607FA440F551F5F3F79F0A3
:102F6000AA27A51708F051E04795880F991F9F3FA2
:102F700031F0BB27B91708F091E0879508959F912C
:102F80009F911124E3CF66277727882799270895F3
:102F900097FBEBDF992329F05F3F29F0552319F0C8
:102FA0000AF4F1CFD3CF940F151E01F4B7CF592FE8
:102FB000482F372F262FCDDF01D0B0CF992339F0FE
:102FC000552329F09F575F57950F13F4CAF1DECFB1
:102FD00091589F3FE1F3A62F00241124BB276627B9
:102FE0005527F8E0A69520F4020E131EB41F651FA6
:102FF000220F331F441F551FFA95A1F7F8E0E72F62
:103000007727F8E0E69520F4130EB41F651F7A1FAA
:10301000330F441F551FAA1FFA95A1F7F82F8827D1
:10302000F69520F4B40F651F7A1F8E1F440F551FAD
:10303000AA1FEE1FFF23A1F788231AF4939539F4F2
:1030400085CF000C111CBB1F661F771F881F01282E
:103050000895552371F1992362F059F15F934F93CD
:103060003F932F93BBD02F913F914F915F91A3DF5F
:1030700025C09F938F937F936F935F934F933F935D
:103080002F93952F842F732F622FFADED7DD9115A2
:103090008105710561052F913F914F915F916F916E
:1030A0007F918F919F9121F09F775058E2DF505888
:1030B0004DCF9FE380E8772766270895092E99234F
:1030C0004AF052E441EB32E7683173078407950711
:1030D00058F03CCF9F7752E44EEA3CEA60357307E4
:1030E0008407950708F04FCF0F925FE348EB3AEA69
:1030F0002BE361DFFF92EF92DF92CF9250E04CE042
:1031000096D0E4E5F0E01ED05F2D4E2D3D2D2C2D08
:10311000CF90DF90EF90FF90FEE94595441F551F3B
:10312000F51B5527406804C0469537952795579558
:10313000FA95D2F7452F550F550B2ADF0F9007FC54
:10314000C0CD0895092E11DFFF92EF92DF92CF924A
:10315000BF92AF92B02CC92ED82EE72EF62EA59096
:1031600018D0A590AA2071F09F938F937F936F93AF
:103170006F2D7E2D8D2D9C2D0CD02F913F914F9139
:103180005F91AADDAF90BF90CF90DF90EF90FF905E
:10319000C5CE7ED047FB406804C02F2D3E2D4D2D5F
:1031A0005C2DEF93FF930ADFFF91EF9171D0AA2777
:1031B00007F80B24102C042607FA4068FF9343DD20
:1031C000FF91992341F0882332F09A95BB0F661F37
:1031D000771F881FF8CFAA9401F7089597FDB6CE00
:1031E000C4DE992309F4B2CEFF92EF92DF92CF9220
:1031F000C92E9FE38F77E2E7F0E0A4DF0C2CC92E05
:10320000D82EE72EF62E602D6E57770B872F972F2F
:1032100054DE5FE341E332E728E1CDDE5C2D4D2D46
:103220003E2D2F2DCF90DF90EF90FF9008CD97FB94
:103230009CDECF93DF93D52FC42F55274427332708
:1032400022279923D9F09F37C8F0F92F67DE592F2D
:10325000482F372F262FF63968F412DE2EDEC030C5
:10326000CD0721F069937993899399939058DF91D1
:10327000CF91E5CC9927882777276627C030CD07DF
:1032800021F02993399349935993DF91CF9146CEF9
:1032900055914591359125910895629FD001739F75
:1032A000F001829FE00DF11D649FE00DF11D929FE2
:1032B000F00D839FF00D749FF00D659FF00D992721
:1032C000729FB00DE11DF91F639FB00DE11DF91F45
:1032D000BD01CF0111240895991B79E004C0991F05
:1032E000961708F0961B881F7A95C9F78095089560
:1032F00097FB092E07260AD077FD04D027D006D0E9
:1033000000201AF4709561957F4F0895F6F7909517
:1033100081959F4F089597FB092E05260ED057FDE6
:1033200004D028D00AD0001C38F450954095309530
:1033300021953F4F4F4F5F4F0895F6F79095809539
:10334000709561957F4F8F4F9F4F0895AA1BBB1BB0
:1033500051E107C0AA1FBB1FA617B70710F0A61B95
:10336000B70B881F991F5A95A9F780959095BC01B6
:10337000CD010895A1E21A2EAA1BBB1BFD010DC0B1
:10338000AA1FBB1FEE1FFF1FA217B307E407F50715
:1033900020F0A21BB30BE40BF50B661F771F881FF1
:1033A000991F1A9469F760957095809590959B0187
:0833B000AC01BD01CF0108953D
:1033B800010204080A14285000051602000F201103
:1033C8002E1F1F2E11202122232425262728050001
:0A33D8000A00007800003CE8030042
:0200000400807A
:0101A200025A
:00000001FF
